Archive member included because of file (symbol)

c:/winavr-20081205/bin/../lib/gcc/avr/4.3.2/avr51\libgcc.a(_udivmodhi4.o)
                              Ex3_1_TFT43_RdReg_Touch.o (__udivmodhi4)
c:/winavr-20081205/bin/../lib/gcc/avr/4.3.2/avr51\libgcc.a(_exit.o)
                              c:/winavr-20081205/bin/../lib/gcc/avr/4.3.2/../../../../avr/lib/avr51/crtm128.o (exit)
c:/winavr-20081205/bin/../lib/gcc/avr/4.3.2/avr51\libgcc.a(_clear_bss.o)
                              Ex3_1_TFT43_RdReg_Touch.o (__do_clear_bss)

Allocating common symbols
Common symbol       size              file

ft800Gpio           0x1               Ex3_1_TFT43_RdReg_Touch.o
intE                0x2               Ex3_1_TFT43_RdReg_Touch.o
intB                0x2               Ex3_1_TFT43_RdReg_Touch.o
intF                0x2               Ex3_1_TFT43_RdReg_Touch.o
num_cha             0x1               Ex3_1_TFT43_RdReg_Touch.o
fracF               0x2               Ex3_1_TFT43_RdReg_Touch.o
fracC               0x2               Ex3_1_TFT43_RdReg_Touch.o
fracD               0x2               Ex3_1_TFT43_RdReg_Touch.o
fracB               0x2               Ex3_1_TFT43_RdReg_Touch.o
intA                0x2               Ex3_1_TFT43_RdReg_Touch.o
intD                0x2               Ex3_1_TFT43_RdReg_Touch.o
fracE               0x2               Ex3_1_TFT43_RdReg_Touch.o
fracA               0x2               Ex3_1_TFT43_RdReg_Touch.o
intC                0x2               Ex3_1_TFT43_RdReg_Touch.o

Memory Configuration

Name             Origin             Length             Attributes
text             0x00000000         0x00020000         xr
data             0x00800060         0x0000ffa0         rw !x
eeprom           0x00810000         0x00010000         rw !x
fuse             0x00820000         0x00000400         rw !x
lock             0x00830000         0x00000400         rw !x
signature        0x00840000         0x00000400         rw !x
*default*        0x00000000         0xffffffff

Linker script and memory map

Address of section .data set to 0x800100
LOAD c:/winavr-20081205/bin/../lib/gcc/avr/4.3.2/../../../../avr/lib/avr51/crtm128.o
LOAD Ex3_1_TFT43_RdReg_Touch.o
LOAD c:/winavr-20081205/bin/../lib/gcc/avr/4.3.2/avr51\libgcc.a
LOAD c:/winavr-20081205/bin/../lib/gcc/avr/4.3.2/../../../../avr/lib/avr51\libc.a
LOAD c:/winavr-20081205/bin/../lib/gcc/avr/4.3.2/avr51\libgcc.a

.hash
 *(.hash)

.dynsym
 *(.dynsym)

.dynstr
 *(.dynstr)

.gnu.version
 *(.gnu.version)

.gnu.version_d
 *(.gnu.version_d)

.gnu.version_r
 *(.gnu.version_r)

.rel.init
 *(.rel.init)

.rela.init
 *(.rela.init)

.rel.text
 *(.rel.text)
 *(.rel.text.*)
 *(.rel.gnu.linkonce.t*)

.rela.text
 *(.rela.text)
 *(.rela.text.*)
 *(.rela.gnu.linkonce.t*)

.rel.fini
 *(.rel.fini)

.rela.fini
 *(.rela.fini)

.rel.rodata
 *(.rel.rodata)
 *(.rel.rodata.*)
 *(.rel.gnu.linkonce.r*)

.rela.rodata
 *(.rela.rodata)
 *(.rela.rodata.*)
 *(.rela.gnu.linkonce.r*)

.rel.data
 *(.rel.data)
 *(.rel.data.*)
 *(.rel.gnu.linkonce.d*)

.rela.data
 *(.rela.data)
 *(.rela.data.*)
 *(.rela.gnu.linkonce.d*)

.rel.ctors
 *(.rel.ctors)

.rela.ctors
 *(.rela.ctors)

.rel.dtors
 *(.rel.dtors)

.rela.dtors
 *(.rela.dtors)

.rel.got
 *(.rel.got)

.rela.got
 *(.rela.got)

.rel.bss
 *(.rel.bss)

.rela.bss
 *(.rela.bss)

.rel.plt
 *(.rel.plt)

.rela.plt
 *(.rela.plt)

.text           0x00000000     0x17e6
 *(.vectors)
 .vectors       0x00000000       0x8c c:/winavr-20081205/bin/../lib/gcc/avr/4.3.2/../../../../avr/lib/avr51/crtm128.o
                0x00000000                __vectors
                0x00000000                __vector_default
 *(.vectors)
 *(.progmem.gcc*)
 *(.progmem*)
                0x0000008c                . = ALIGN (0x2)
                0x0000008c                __trampolines_start = .
 *(.trampolines)
 .trampolines   0x0000008c        0x0 linker stubs
 *(.trampolines*)
                0x0000008c                __trampolines_end = .
 *(.jumptables)
 *(.jumptables*)
 *(.lowtext)
 *(.lowtext*)
                0x0000008c                __ctors_start = .
 *(.ctors)
                0x0000008c                __ctors_end = .
                0x0000008c                __dtors_start = .
 *(.dtors)
                0x0000008c                __dtors_end = .
 SORT(*)(.ctors)
 SORT(*)(.dtors)
 *(.init0)
 .init0         0x0000008c        0x0 c:/winavr-20081205/bin/../lib/gcc/avr/4.3.2/../../../../avr/lib/avr51/crtm128.o
                0x0000008c                __init
 *(.init0)
 *(.init1)
 *(.init1)
 *(.init2)
 .init2         0x0000008c        0xc c:/winavr-20081205/bin/../lib/gcc/avr/4.3.2/../../../../avr/lib/avr51/crtm128.o
 *(.init2)
 *(.init3)
 *(.init3)
 *(.init4)
 .init4         0x00000098       0x1c c:/winavr-20081205/bin/../lib/gcc/avr/4.3.2/../../../../avr/lib/avr51/crtm128.o
                0x00000098                __do_copy_data
 .init4         0x000000b4       0x10 c:/winavr-20081205/bin/../lib/gcc/avr/4.3.2/avr51\libgcc.a(_clear_bss.o)
                0x000000b4                __do_clear_bss
 *(.init4)
 *(.init5)
 *(.init5)
 *(.init6)
 *(.init6)
 *(.init7)
 *(.init7)
 *(.init8)
 *(.init8)
 *(.init9)
 .init9         0x000000c4        0x8 c:/winavr-20081205/bin/../lib/gcc/avr/4.3.2/../../../../avr/lib/avr51/crtm128.o
 *(.init9)
 *(.text)
 .text          0x000000cc        0x4 c:/winavr-20081205/bin/../lib/gcc/avr/4.3.2/../../../../avr/lib/avr51/crtm128.o
                0x000000cc                __vector_22
                0x000000cc                __vector_28
                0x000000cc                __vector_1
                0x000000cc                __vector_32
                0x000000cc                __vector_34
                0x000000cc                __vector_24
                0x000000cc                __vector_12
                0x000000cc                __bad_interrupt
                0x000000cc                __vector_6
                0x000000cc                __vector_31
                0x000000cc                __vector_3
                0x000000cc                __vector_23
                0x000000cc                __vector_30
                0x000000cc                __vector_25
                0x000000cc                __vector_11
                0x000000cc                __vector_13
                0x000000cc                __vector_17
                0x000000cc                __vector_19
                0x000000cc                __vector_7
                0x000000cc                __vector_27
                0x000000cc                __vector_5
                0x000000cc                __vector_33
                0x000000cc                __vector_4
                0x000000cc                __vector_9
                0x000000cc                __vector_2
                0x000000cc                __vector_21
                0x000000cc                __vector_15
                0x000000cc                __vector_29
                0x000000cc                __vector_8
                0x000000cc                __vector_26
                0x000000cc                __vector_14
                0x000000cc                __vector_10
                0x000000cc                __vector_16
                0x000000cc                __vector_18
                0x000000cc                __vector_20
 .text          0x000000d0     0x16ea Ex3_1_TFT43_RdReg_Touch.o
                0x00000134                FT800memWrite8
                0x0000042a                Start_CMDOffset
                0x000007e4                Touch_Calibrate
                0x0000012c                FT800_PD_hi
                0x000001c6                FT800memWrite32
                0x000004a0                Start_CMDList
                0x0000023a                FT800memWriteStr
                0x00000130                FT800_PD_lo
                0x0000046c                incCMDOffset
                0x000002ca                FT800memRead8
                0x000000ee                spi_sdo_hi
                0x0000030e                FT800memRead16
                0x000000fa                spi_sck_lo
                0x0000087a                FT800_Initial
                0x00001178                Update_Screen
                0x0000060e                Text_CMD
                0x00000364                FT800memRead32
                0x0000178e                main
                0x000000d0                delay_ms
                0x000000fe                spi_cs_hi
                0x000002b4                FT800_HostCmdWrite
                0x000000f2                spi_sdo_lo
                0x00000106                spi_rw
                0x00000482                End_incCMDOffset
                0x00000178                FT800memWrite16
                0x00000b8e                Conv_hex_to_Ascii
                0x000000f6                spi_sck_hi
                0x0000153e                User_App
                0x00000102                spi_cs_lo
                0x00000580                End_CMDList
                0x000000e4                init_port
 .text          0x000017ba        0x0 c:/winavr-20081205/bin/../lib/gcc/avr/4.3.2/avr51\libgcc.a(_udivmodhi4.o)
 .text          0x000017ba        0x0 c:/winavr-20081205/bin/../lib/gcc/avr/4.3.2/avr51\libgcc.a(_exit.o)
 .text          0x000017ba        0x0 c:/winavr-20081205/bin/../lib/gcc/avr/4.3.2/avr51\libgcc.a(_clear_bss.o)
                0x000017ba                . = ALIGN (0x2)
 *(.text.*)
 .text.libgcc   0x000017ba       0x28 c:/winavr-20081205/bin/../lib/gcc/avr/4.3.2/avr51\libgcc.a(_udivmodhi4.o)
                0x000017ba                __udivmodhi4
 .text.libgcc   0x000017e2        0x0 c:/winavr-20081205/bin/../lib/gcc/avr/4.3.2/avr51\libgcc.a(_exit.o)
 .text.libgcc   0x000017e2        0x0 c:/winavr-20081205/bin/../lib/gcc/avr/4.3.2/avr51\libgcc.a(_clear_bss.o)
                0x000017e2                . = ALIGN (0x2)
 *(.fini9)
 .fini9         0x000017e2        0x0 c:/winavr-20081205/bin/../lib/gcc/avr/4.3.2/avr51\libgcc.a(_exit.o)
                0x000017e2                exit
                0x000017e2                _exit
 *(.fini9)
 *(.fini8)
 *(.fini8)
 *(.fini7)
 *(.fini7)
 *(.fini6)
 *(.fini6)
 *(.fini5)
 *(.fini5)
 *(.fini4)
 *(.fini4)
 *(.fini3)
 *(.fini3)
 *(.fini2)
 *(.fini2)
 *(.fini1)
 *(.fini1)
 *(.fini0)
 .fini0         0x000017e2        0x4 c:/winavr-20081205/bin/../lib/gcc/avr/4.3.2/avr51\libgcc.a(_exit.o)
 *(.fini0)
                0x000017e6                _etext = .

.data           0x00800100      0x186 load address 0x000017e6
                0x00800100                PROVIDE (__data_start, .)
 *(.data)
 .data          0x00800100        0x0 c:/winavr-20081205/bin/../lib/gcc/avr/4.3.2/../../../../avr/lib/avr51/crtm128.o
 .data          0x00800100      0x185 Ex3_1_TFT43_RdReg_Touch.o
                0x0080026b                int_E
                0x0080025b                sig_D
                0x00800255                frac_C
                0x00800271                frac_E
                0x00800231                sig_A
                0x00800233                int_A
                0x0080024f                int_C
                0x00800239                frac_A
                0x0080023f                sig_B
                0x00800263                frac_D
                0x00800269                sig_E
                0x00800241                int_B
                0x0080027f                frac_F
                0x0080024d                sig_C
                0x00800279                int_F
                0x0080025d                int_D
                0x00800277                sig_F
                0x00800247                frac_B
 .data          0x00800285        0x0 c:/winavr-20081205/bin/../lib/gcc/avr/4.3.2/avr51\libgcc.a(_udivmodhi4.o)
 .data          0x00800285        0x0 c:/winavr-20081205/bin/../lib/gcc/avr/4.3.2/avr51\libgcc.a(_exit.o)
 .data          0x00800285        0x0 c:/winavr-20081205/bin/../lib/gcc/avr/4.3.2/avr51\libgcc.a(_clear_bss.o)
 *(.data*)
 *(.rodata)
 *(.rodata*)
 *(.gnu.linkonce.d*)
                0x00800286                . = ALIGN (0x2)
 *fill*         0x00800285        0x1 00
                0x00800286                _edata = .
                0x00800286                PROVIDE (__data_end, .)

.bss            0x00800286       0x22
                0x00800286                PROVIDE (__bss_start, .)
 *(.bss)
 .bss           0x00800286        0x0 c:/winavr-20081205/bin/../lib/gcc/avr/4.3.2/../../../../avr/lib/avr51/crtm128.o
 .bss           0x00800286        0x8 Ex3_1_TFT43_RdReg_Touch.o
                0x0080028a                cmdBufferRd
                0x0080028c                cmdBufferWr
                0x00800286                DL_Offset
                0x00800288                cmdOffset
 .bss           0x0080028e        0x0 c:/winavr-20081205/bin/../lib/gcc/avr/4.3.2/avr51\libgcc.a(_udivmodhi4.o)
 .bss           0x0080028e        0x0 c:/winavr-20081205/bin/../lib/gcc/avr/4.3.2/avr51\libgcc.a(_exit.o)
 .bss           0x0080028e        0x0 c:/winavr-20081205/bin/../lib/gcc/avr/4.3.2/avr51\libgcc.a(_clear_bss.o)
 *(.bss*)
 *(COMMON)
 COMMON         0x0080028e       0x1a Ex3_1_TFT43_RdReg_Touch.o
                0x0080028e                ft800Gpio
                0x0080028f                intE
                0x00800291                intB
                0x00800293                intF
                0x00800295                num_cha
                0x00800296                fracF
                0x00800298                fracC
                0x0080029a                fracD
                0x0080029c                fracB
                0x0080029e                intA
                0x008002a0                intD
                0x008002a2                fracE
                0x008002a4                fracA
                0x008002a6                intC
                0x008002a8                PROVIDE (__bss_end, .)
                0x000017e6                __data_load_start = LOADADDR (.data)
                0x0000196c                __data_load_end = (__data_load_start + SIZEOF (.data))

.noinit         0x008002a8        0x0
                0x008002a8                PROVIDE (__noinit_start, .)
 *(.noinit*)
                0x008002a8                PROVIDE (__noinit_end, .)
                0x008002a8                _end = .
                0x008002a8                PROVIDE (__heap_start, .)

.eeprom         0x00810000        0x0
 *(.eeprom*)
                0x00810000                __eeprom_end = .

.fuse
 *(.fuse)
 *(.lfuse)
 *(.hfuse)
 *(.efuse)

.lock
 *(.lock*)

.signature
 *(.signature*)

.stab
 *(.stab)

.stabstr
 *(.stabstr)

.stab.excl
 *(.stab.excl)

.stab.exclstr
 *(.stab.exclstr)

.stab.index
 *(.stab.index)

.stab.indexstr
 *(.stab.indexstr)

.comment
 *(.comment)

.debug
 *(.debug)

.line
 *(.line)

.debug_srcinfo
 *(.debug_srcinfo)

.debug_sfnames
 *(.debug_sfnames)

.debug_aranges  0x00000000       0x20
 *(.debug_aranges)
 .debug_aranges
                0x00000000       0x20 Ex3_1_TFT43_RdReg_Touch.o

.debug_pubnames
                0x00000000      0x39e
 *(.debug_pubnames)
 .debug_pubnames
                0x00000000      0x39e Ex3_1_TFT43_RdReg_Touch.o

.debug_info     0x00000000     0x1110
 *(.debug_info)
 .debug_info    0x00000000     0x1110 Ex3_1_TFT43_RdReg_Touch.o
 *(.gnu.linkonce.wi.*)

.debug_abbrev   0x00000000      0x27e
 *(.debug_abbrev)
 .debug_abbrev  0x00000000      0x27e Ex3_1_TFT43_RdReg_Touch.o

.debug_line     0x00000000     0x105b
 *(.debug_line)
 .debug_line    0x00000000     0x105b Ex3_1_TFT43_RdReg_Touch.o

.debug_frame    0x00000000      0x200
 *(.debug_frame)
 .debug_frame   0x00000000      0x200 Ex3_1_TFT43_RdReg_Touch.o

.debug_str      0x00000000      0x442
 *(.debug_str)
 .debug_str     0x00000000      0x442 Ex3_1_TFT43_RdReg_Touch.o
                                0x491 (size before relaxing)

.debug_loc      0x00000000      0x958
 *(.debug_loc)
 .debug_loc     0x00000000      0x958 Ex3_1_TFT43_RdReg_Touch.o

.debug_macinfo
 *(.debug_macinfo)
OUTPUT(Ex3_1_TFT43_RdReg_Touch.elf elf32-avr)
LOAD linker stubs

.debug_ranges   0x00000000       0x60
 .debug_ranges  0x00000000       0x60 Ex3_1_TFT43_RdReg_Touch.o
